:100000000EC01DC01CC01BC01AC019C018C017C02C
:1000100016C015C014C013C012C011C010C01124E6
:100020001FBECFE5D1E0DEBFCDBF20E0A0E6B0E04F
:1000300001C01D92A536B207E1F788D023C1E0CFF9
:10004000FC019081862F809598239083ABECB0E0E3
:100050001197F1F700C00000908140FF02C0962B7D
:1000600001C098239083ABECB0E01197F1F700C08A
:100070000000908141FF02C0962B01C0982390831D
:10008000ABECB0E01197F1F700C00000908142FFA7
:1000900002C0962B01C098239083ABECB0E011977F
:1000A000F1F700C00000908143FF02C0962B01C011
:1000B00098239083ABECB0E01197F1F700C00000FB
:1000C000908144FF02C0962B01C098239083ABEC33
:1000D000B0E01197F1F700C00000908145FF02C029
:1000E000962B01C098239083ABECB0E01197F1F709
:1000F00000C00000908146FF02C0962B01C09823EB
:100100009083ABECB0E01197F1F700C0000047FF1F
:1001100004C08081862B808303C0908198239083C4
:100120008BEC90E00197F1F700C000008081862BF6
:100130008083ABECB0E01197F1F700C000008BECCE
:1001400090E00197F1F700C00000089580E886BDB7
:1001500016BCC29ABA9AC39ABB9A82E087B984E85D
:1001600086B910926400109263001092620010929F
:1001700061001092600080916000843630F5C39A6F
:10018000369A3699FECF24B135B1809161009091B5
:100190006200820F931F9093620080936100C39866
:1001A000369A3699FECF24B135B180916300909193
:1001B0006400820F931F909364008093630080918A
:1001C00060008F5F80936000D6CF41E064E088E3F9
:1001D00090E036DF8FEC97E00197F1F700C0000068
:1001E00042E064E088E390E02BDF8FEC97E001973A
:1001F000F1F700C0000043E064E088E390E020DF16
:100200008FEC97E00197F1F700C0000044E064E054
:1002100088E390E015DF8FEC97E00197F1F700C0DD
:1002200000004091630064E088E390E009DF8FEC18
:1002300097E00197F1F700C000004091640064E08E
:1002400088E390E0FDDE8FEC97E00197F1F700C0C6
:1002500000004091610064E088E390E0F1DE8FEC03
:1002600097E00197F1F700C000004091620064E060
:1002700088E390E0E5DE8FEC97E00197F1F700C0AE
:0802800000006FCFF894FFCFDE
:00000001FF
